:040E820021D6007005
:040E86002572006F62
:040E8A0024D0005E12
:040E8E0023B7007016
:040E920037B700531B
:100FF800E527C4030354037870F6FC25E025E024B4
:101008004FF582E43448F583120E4CE87871120EDD
:1010180002E5270303035407FC7870F6B407193078
:10102800380678BE7601800D30390678BE760180A4
:101038000478BE76010210E6B4060778BE76000290
:1010480010E690485B93FCE4FDFEFF08120469E497
:10105800FAFB7820794E740312033A700678BE764C
:1010680005807B78107927740312033A700678BEDE
:101078007600806A791D784C740312033A700678FA
:10108800BE7601805979177870740312033A700696
:1010980078BE7601804879137888740312033A7011
:1010A8000678BE76018037790F78A0740312033A68
:1010B800700678BE76028026790B78B8740312031E
:1010C8003A700678BE76038015790978C4740312DD
:1010D800033A700678BE7603800478BE760422D27E
:1010E80009D312441C1218AD7C051216467C011255
:1010F8001646121C891220E6400280F912214A780D
:10110800A1ECF6700280F57C401237A178A1E6B414
:101118000F077C07121646801DB40C077C031216B5
:10112800468013B40D04C209800CB40E077C01126A
:10113800164680028000121C892009B97D967E0E11
:101148007F02121CB27C1012377D121E70D322123D
:1011580037B77CFF02377DAC4BAD4AAE49AF48127A
:10116800098F7870120DEAA82FA92EAA2DAB2C1280
:1011780005817870120E30120581120DA278701256
:101188000E24A833A932AA31AB30120581120DC63C
:10119800120833A837A936AA35AB34120833787445
:1011A800120DEAA83BA93AAA39AB381205811209EF
:1011B800308C4B8D4A8E498F48227882ECF6122B60
:1011C800EC4002C3227882E614700312115F78B8EB
:1011D800E67881F6AC4BAD4AAE49AF48A83FA93E88
:1011E800AA3DAB3C740312033A700F1203DD787DFD
:1011F800120DEA08C64408F680141203EE787D1230
:101208000DEA0808E66403600518C654F7F6788105
:10121800E678B8F67882E66403600C787C760B781A
:101228007D120E24121DABD322E54F454E454D4588
:101238004C700C854B4F854A4E85494D85484CACC2
:101248004BAD4AAE49AF48A84FA94EAA4DAB4C7416
:101258000712033A70051203DD80031203EE78D6F5
:10126800120DEAE4F9FAFB7814740712033A7021B4
:101278007D9D7E0E7F02121CB2121157C205E4F545
:1012880043F542F541F540F54FF54EF54DF54C80E7
:101298001BAC4BAD4AAE49AF48784012042F854B82
:1012A8004F854A4E85494D85484CD205A20522C234
:1012B80007C208E4F543F542F541F5407883760026
:1012C800080876003007030213607C031211C2403D
:1012D8004112214A7884ECF6700280E87C6012376B
:1012E800A17884E6B40A028003B40C127DA47E0EB1
:1012F8007F02121CB27C8F12377DD208800BB40D8E
:1013080008D2077883760280001220E6400280F92E
:1013180080B220080280AD1212315026787C760BFC
:101328007885E67D00FCE4FF7409C39CFCEF9DFD15
:101338003395E0FFFE121DAB7C1F12377D788506C2
:10134800800AD20778857600181876017885E62411
:10135800F65002D2070212CC7840E4FDFEFF7C0A68
:101368001204697883E6FC227887120DD81212B726
:101378007886ECF6600122AC43AD42AE41AF40E462
:10138800FAFB78307975740712033A70107DAB7EDA
:101398000E7F02121CB212115778867601AC43AD4B
:1013A80042AE41AF407887120E1B120D317886E6A7
:1013B800FC227887120DD81212B77886ECF66001F5
:1013C80022AC43AD42AE41AF4008120E1B120D31A4
:1013D8007886E6FC22788B120DEA1212B77886EC32
:1013E800F6600122AC43AD42AE41AF40E4FB7A0364
:1013F800790D7840740312033A70107DB27E0E7F27
:1014080002121CB212115778867601121C6F788767
:10141800120DEAA843A942AA41AB40740F12033A3D
:101428007014788B120E24A843A942AA41AB4074C9
:101438000712033A70107DB97E0E7F02121CB21299
:10144800115778867601AC43AD42AE41AF40788FF4
:10145800120E1B120D317886E6FC22787D120DEAF9
:10146800121C6F12098F7879120DEA7881120E24F6
:10147800787D120E301203DD12098F120DA27879D1
:10148800120E24E4F8F9FA7B3F120581120DC612F8
:1014980006FF7875120DEA7885120E24787D120EF3
:1014A800301203DD12098F7879120E301206F378A4
:1014B80075120E30120826120DA27879120E24E445
:1014C800F8F9FA7B3F120581120DC61206F38C2F2C
:1014D8008D2E8E2D8F2C787D120E2408120E301230
:1014E80003CD12098FA82FA92EAA2DAB2C12058186
:1014F800EE4F6004EF6480FF7875120E30120833E7
:101508008C338D328E318F30787D120E2412098FF4
:10151800A82FA92EAA2DAB2C1205817881120E3086
:101528001209EB120581787D120E301209EB120DAB
:10153800A2120DB47875120E24120DC6120581126E
:101548000DC612081A787D120E301209EB120833F4
:101558008C378D368E358F34E4F53BF53A75383F48
:10156800753980787D120E2412098F7A807B3F129C
:1015780005737875120DEA12093078BF120DEA78F2
:1015880071763F08E4F608F608F622C2077884EC7C
:10159800F62007737884E6FC1211C2500280F2121A
:1015A800214A7883ECF6700280E77C601237A178D4
:1015B80083E6120BBB15D60715E50915F40A15F4D1
:1015C8000C15F80D15D60E15E50F0000160678381F
:1015D8007CAC7DC57EA77F37120A8A802178387C4B
:1015E800AC7DC57EA77F37120A858012D207800E90
:1015F800854B3F854A3E85493D85483C8000122001
:10160800E6400280F9808A7C00227E047DAC7C075B
:10161800121FDD78BF120E2412098F78C3120E3004
:101628001206FFA83BA93AAA39AB3812058178708F
:10163800120DEA12093078BF020DEA021F08D21A09
:10164800D21178A0ECF6AC3BAD3AAE39AF38743372
:10165800F8F9FA7B3F7403120A35700F7B3F746602
:10166800F9F87AA67407120A35700BE4F53BF53AD7
:1016780075383F753980122BEC400280F978A0E666
:10168800B40109121E70789276008018B4030678A7
:10169800927601800FB405067892760680067892D5
:1016A800760780001220E6400280F978A0E61470E0
:1016B8000312115F30201478A0E6B4030E854B3F67
:1016C800854A3E85493D85483C8009E4F53FF53E1D
:1016D800F53DF53C854B4F854A4E85494D85484C2F
:1016E8007892E624F95003021840121C897892E691
:1016F800120B8500061831170D1730175C17911754
:10170800CE17EC180F7DC07E0E7F02121CB27C9F94
:1017180012377D7C011215937893ECF61216127825
:1017280092C62404F60218317DC77E0E7F02121C71
:10173800B27C9F12377D7C9F12377D7C9F12377D4C
:101748007C9F12377D7D94E4FEFF1213707893EC32
:10175800F6021831E4F54FF54EF54DF54C7DCE7E89
:101768000E7F02121CB27C9F12377D7C9F12377D40
:101778007C9F12377D7C9F12377D7D98E4FEFF1297
:1017880013BA7893ECF6021831E4F54FF54EF54D9F
:10179800F54C7DD57E0E7F02121CB27C9F12377DE0
:1017A8007C9F12377D7C9F12377D7C9F12377DE4AA
:1017B800788FF608F608769C7894120E241213DDBA
:1017C8007893ECF68063789C120E247985120DF6D6
:1017D8007898120E247981120DF67894120E24123C
:1017E800146380451216437DDC7E0E7F02121CB204
:1017F8007CFF1237A17C9F12377D7C9F12377D12A8
:101808001C897892068022E4F54FF54EF54DF54C8B
:101818007DE37E0E7F02121CB27C9F12377D7C0511
:101828001215937893ECF680007893E6B402028060
:1018380007700218060216E8C211227873EEF6182D
:1018480018EDF608ECF6EEB402180808120E1BEEB6
:101858007F00120D97FEFAEFFB1201367970E8F758
:10186800804125E0FAE433FBEDC0E0ECC0E0787499
:10187800120E12ED2AFDEE3BFE90FFFE120C26FA28
:10188800D0E0FDD0E0CDFC120194E8FAE9FB7874D1
:10189800120E127873E67900120D8CF81201417954
:1018A80070E8F7FC2278779047A9790C120D86D258
:1018B80011C2067E027DA47C07121FDD78C3E6FDF7
:1018C80008E678B276FFFC9047E5E493547F78B356
:1018D800F67887EDF608ECF608EDF608ECF60876EB
:1018E80000788476027887E6FD08E6FC7884E6FFCF
:1018F800EF24FA4057EF25E02477F8ECFAEDFBE601
:10190800F908E6F8120141EF25E024777985C8F750
:10191800FEE4FBEFF9EBFFE6FB08E6FAEDC0E0ECCE
:10192800C0E0E9FC120116D0E0FFD0E0CFC398FE7A
:10193800EF99CCFDCCCDFAEEFCEAFF7885E690472E
:10194800DC93FEEF24B2F8EEF60F80A47887EDF66C
:1019580008ECF67884EFF67889E6FD08E6FC7B0368
:101968007AE81201367985E8F70909EDF709ECF705
:101978007F027884EFF61220E6400280F9C2053033
:101988000503021AFC12214A7883ECF6600C7C608D
:101998001237A11220E6400280F9E52A249B500F55
:1019A80030060C788B06E624FA50027600C206E56B
:1019B8002A24CE4002D206788BE624FD500474FF18
:1019C80080077885E69047DC93FC7884E624B2F8B3
:1019D800ECF67883E6C3940C406BB40200B3406520
:1019E800E47874F608F60876777887E6FD08E6FC6A
:1019F8007884E6FE1218437884E625E02477080800
:101A0800CCF6CC7D00F8E6FB08E6FA12011DE8FCEE
:101A1800E9FD7888C3E69CF618E69DF67884E62505
:101A2800E02477FC08E67F00FEECF8E6FB08E6FA1F
:101A3800120116E8FCE9FD7888E62CF618E63DF672
:101A4800D205021AF9B402028003021AEAE4787491
:101A5800F608F60876777887E6FD08E6FC7884E6E7
:101A6800FE1218437884E625E024770808CCF6CCE3
:101A78007D00F8E6FB08E6FA12011DE8FCE9FD78AE
:101A880088C3E69CF618E69DF67884E625E0247778
:101A9800FC08E67F00FEECF8E6FB08E6FA12011601
:101AA800E8FCE9FD7888E62CF618E63DF6EE904766
:101AB800DC93FC7884E624B2F8ECF6788406E62415
:101AC800FA50027602E47874F608F6087677788792
:101AD800E6FD08E6FC7884E6FE1218437885ECF605
:101AE800800FB4030C788506E624F6500276008051
:101AF80000021987C2117889E6FD08E61818667091
:101B080005ED1866606D7887E6FD08E679C4F7ED9F
:101B180019F77E027DA47C07121FB97889E6FD08B3
:101B2800E6FC120979E4F87B477AAF79C8120833E2
:101B38007887E6F908E6F81209CB120DA2E4FC7FD3
:101B4800477EAF7DC8120833120DC61206F3788C93
:101B5800120DEA7838120A8F78BF120E2412098FF4
:101B6800788C120E3012058112093078BF120DEAF6
:101B7800121F0822121C897E027DA47C07121FDD19
:101B880078C3E6FD08E67872CDF6CD08F6D3940F53
:101B9800ED9427400518E4F608F6E6FC18E6FDE49F
:101BA800FEFFFB04FA795F78901203CD7878120D66
:101BB800EA7E027DB27C07121FDD78C3E6FD08E6E7
:101BC8007872CDF6CD08F6D3940FED94274005181A
:101BD800E4F608F6E6FC18E6FDE4FEFFFB04FA79F5
:101BE8005F78901203CD7874120DEA7874120E247F
:101BF80008120E30740512033A706B7872E6FD080D
:101C0800E678C8F6ED18F67E027DA47C07121FB9A7
:101C1800787CA63808A63908A63A08A63B78781230
:101C28000E2412098F7874120E301209EB1206FF77
:101C38007838120A8F78BF120E301209EB120DB4E1
:101C4800787C120E24120DC61206F3A83BA93AAAF4
:101C580039AB38120581787C120DEA12093078BF49
:101C6800120DEA121F0822E527C4030354037870F3
:101C7800F625E025E0244FF582E43448F583020E8A
:011C88003C1F
:100E960020202020202000554E5354424C00205341
:100EA6005441424C00484848484848002053415461
:100EB6005552004C4C4C4C4C4C005452494D202041
:100EC60000554E4C4F4144002035305045520031BC
:100ED6003030504552002020454E442000434845BE
:040EE600434B20005A
:0C47A90086A0271003E80064000A00014D
:101C890078B27A0774FFF608DAFC7A0722121C89FF
:101C990078B8E67853F678B9E620E3067853C6446F
:101CA90009F67853E678B8F6227852760008120DCC
:101CB900D87852E624FA402508120E12120BE424B1
:101CC900E090481493FC7852E624B2F8ECF60DED56
:101CD90070010E7853120DD878520680D42278B943
:101CE900E654079047D793540FF424067855F6C263
:101CF90000C201785AEDF608ECF612097978561205
:101D09000DEAA21A500474BF800274FF78B2F67803
:101D19005276017852E624FA5003021DAAE625E01C
:101D290025E024B5F582E43447F583120E3C785654
:101D3900120E301206F31209307853ECF6120972BA
:101D490018E625E025E024B5F582E43447F5831249
:101D59000E4C1205817856120A8A7852E678556631
:101D6900700BD2007852E624FB4002D20120000514
:101D79007853E660107853E69047DC9308F6200024
:101D890002D20080030876FF300106C6547FF6C2EE
:101D990001E6FC1818E624B2F8ECF6785206021DA2
:101DA9001C227878120DEA08E6B40B0C301103E412
:101DB900800378B9E67870F67870E654079047D7CB
:101DC90093540FF424067873F6C205C20612098FDC
:101DD90008120DEA787076007870E624FA5003024A
:101DE9001E6FE625E025E024B5F582E43447F58346
:101DF900120E3C7874120E301206F3120930787103
:101E0900ECF612097218E625E025E024B5F582E41E
:101E19003447F583120E4C1205817874120A8A78B8
:101E290070E6787366700BD2057870E624FB400281
:101E3900D2062005057871E660107871E69047DCD6
:101E49009308F6200502D20580030876FF300606BE
:101E5900C6547FF6C206E6FC1818E624B2F8ECF67A
:071E6900787006021DE12262
:1047B50047C35000461C4000447A000042C8000030
:0847C500412000003F800000CC
:101E70007E047DA07C07121FDD78C3E6F52708E607
:101E8000F52808E6FC08E678B9F67862ECF67E08F4
:101E90007DA87C07121FDD78C3120E2478BF120DB7
:101EA000EA78C7120E248C3B8D3A8E398F387E0823
:101EB0007DB07C07121FDD78C3120E248C2F8D2E6F
:101EC0008E2D8F2C08120E248C338D328E318F3054
:101ED0007E047DB87C07121FDD78C3120E248C3778
:101EE0008D368E358F347862E66427601A752788C0
:101EF00075284178B9760178C3761F08763A7E0254
:101F00007DA47C07121FB9227E027DA47C07121FCC
:101F1000DD78C3E6FD08E618A627FCE52808F608E4
:101F2000762778B9E678C6F608EDF608ECF678700C
:101F3000EDF608ECF67E087DA07C07121FB97E083E
:101F40007DC07C07121FB978BF120E2478C3120D12
:101F5000EAAC3BAD3AAE39AF3808120DEA7E087DE7
:101F6000A87C07121FB97E087DC87C07121FB978AC
:101F7000C3A62C08A62D08A62E08A62FAC33AD327A
:101F8000AE31AF3008120DEA7E087DB07C07121F1B
:101F9000B97E087DD07C07121FB978C3A63408A685
:101FA0003508A63608A6377E047DB87C07121FB90F
:101FB0007E047DD87C07021FB9E4785CF608F60839
:101FC00076C37861EEF618EDF618ECF6785BEEF66F
:101FD000785C120E1B7858120DE10246EFE4785C33
:101FE000F608F60876C37861EEF618EDF618ECF60A
:101FF000785BEEF6785C120E1B7858120DE1024702
:01200000409F
:10200100C0E0C082C083C0D075D018758CFCE58A51
:10201100B414050000008015B413040000800EB450
:102021001203008008B411028003008000758A3910
:10203100B20B300B2E052BE52B700F53883F758D9E
:1020410000758B00C296C2258019308F07202504A8
:10205100D225C28FB4BD05752BFF8007B43204D2DF
:1020610096D28E0526E52624F85003752600E5262E
:102071009047FC93F323F323F323F323F323F32375
:10208100F323F3FCE52690480493F323F323F3238E
:10209100F323F323F323F323F3FCE52690480C9376
:1020A100F323F323F323F323F323F323F323F3782A
:1020B10050F6E526B4070474FF8005FC24B2F8E667
:1020C1007850F6F223F223F223F223F223F223F2E1
:1020D10023F2D2A6C2A7052AD2A7C2A6D0D0D08306
:0520E100D082D0E032C6
:03000B00022001CF
:1020E600C20078527600E5267057E526785266706B
:1020F6000280F7E6FE7F00EF24EC4011EE652660D5
:102106000280F9EE6526700280F90F80EA7852EEB9
:10211600F608EFF67F00EF24FD401D7E00EE6526F3
:10212600700280F9AE26EE600CAE26E5A0540F6074
:1021360002C32280F10F80DE7853EFF618EEF6D256
:1021460000A200227852A626087600087600E5A0AE
:10215600540F6064E526181866705DE526785266A9
:10216600700280F7E526785266600280F7E52678E9
:102176005266700280F7E526785266600280F7E5BF
:10218600A0540F08F6E6603030E0050876008013AC
:1021960030E105087601800B30E2050876028003FF
:1021A6000876031818E6B407037403F6E625E02557
:1021B600E008084618F6D21E7853E6FC221220E6FE
:1021C600400280F912214A7870ECF6700280F522FE
:1021D600121C89C201786976000876000876000824
:1021E600E4F608F608F608F6123D3DECB4050612CC
:1021F60041A00223AE7C401237A1C2AC1220E640B9
:102206000280F912214A7868ECF6700280F5B40C67
:102216000A7C601237A1D2010223AEB410028003F9
:102226000223607C601237A1786C120E24E4FB0452
:10223600FA79407851740D12033A600302235E7DE9
:10224600EA7E0E7F02121CB278C3E4F608F608F6A0
:1022560008F608F608F608F608F6786A7600786A48
:10226600E624F65003022343E675F00AA478C37603
:1022760000087600786BF6FD7E027C00121FB978A6
:10228600C3E4F608F6786BE62402FD7E027C0012B3
:102296001FB978C37600786BE62404FD7E017C00C6
:1022A600121FB97C1F12377D78C3E4F608F608F6CC
:1022B60008F6786BE6FD7E047C01121FB978C3E44C
:1022C600F608F6786BE62404FD7E027C01121FB93F
:1022D60078C3E4F608F6786BE62406FD7E027C01F8
:1022E600121FB978C37600786BE62408FD7E017C60
:1022F60001121FB97C1F12377D78C3E4F608F60871
:10230600F608F6786BE6FD7E047C02121FB978C3E8
:10231600E4F608F6786BE62404FD7E027C02121FC2
:10232600B978C37600786BE62406FD7E017C02123E
:102336001FB97C1F12377D786A060222647CFF1261
:1023460037A17C601237A17DF17E0E7F02121CB28E
:102356007CFF12377D121C89804E24F6404A7C6031
:102366001237A1786906786C120E24E4F9FAFB7824
:102376000A1201B67868E6F8E4F9FAFB1203CD789A
:102386006C120DEA7869E624FA5014121C897868F2
:10239600E6FCE4FDFEFF786C120DEA78697601E64C
:1023A600F424B32406F876BF2001030221EED20CF2
:1023B60022200F030237B778D6E6084608460846B5
:1023C60060030237B7C2017C0212365F5018854B94
:1023D6003F854A3E85493D85483C78D47600C20F04
:1023E60078D3760080031237B722E527C403035457
:1023F600037852F6FC25E025E0244FF582E43448C4
:10240600F583120E4CE5270303035407FCE87856C0
:10241600120E027852ECF6E527540708F6EC9048BF
:102426005B93F8E4F9FAFB120E6B7856120469789E
:1024360052E6B40729ECFAEDFB08E61490486393DC
:10244600F8120121E8FAE9FB7853E6937900F8C31C
:10245600EA98FAEB997854F608CAF6CA8053B40695
:102466002AECFAEDFB08E624FE90486393F8120185
:1024760021E8FAE9FB7853E6937900F8C3EA98FA7B
:10248600EB997854F608CAF6CA8026ECFAEDFB08F2
:10249600E690486393F8120121E8FAE9FB7853E6DF
:1024A600937900F8C3EA98FAEB997854F608CAF6D5
:1024B600CAFDEAFC2278D6E4F608F608F608F630F5
:1024C6002302C223302402C22422200F030237B77C
:1024D600AC4BAD4AAE49AF48A83FA93EAA3DAB3C7E
:1024E600740712033A70051203DD80031203EE78B7
:1024F6005A120DEA78BEE690488393F8E4F9FAFB9F
:10250600740F12033A70051224BB805F78D6E60872
:1025160046084608466008300D030224BB80063094
:102526001A030237B71223F0E4FEFFA847A946AA0A
:1025360045AB44740B12033A70030237B7AC4BAD8C
:102546004AAE49AF48A83FA93EAA3DAB3C74071224
:10255600033A70141203DD78D6120DEA302302C254
:1025660023302402C22480031237B72230410D30B3
:10257600460512258E80031237B7800B30400512B0
:10258600264380031237B722204203022618B21CC4
:10259600301C12C2167DF87E0E7F02121CB27CFF22
:1025A60012377D80647DFF7E0E7F02121CB27CFF97
:1025B60012377D123A967C0C7D067E0F7F02123A08
:1025C600D3A21A9202A228921A7866760B78BA12C9
:1025D6000E24123BD4A202921A30180D7C047D13ED
:1025E6007E0F7F02123AD3801B30440D7C047D1887
:1025F6007E0F7F02123AD3800B7C047D1D7E0F7FF7
:1026060002123AD37C01123BB57CFF12377DD217FA
:10261600802AB21C301C107DF87E0E7F02121CB27E
:102626007CFF12377D800E7DFF7E0E7F02121CB26C
:102636007CFF12377D7CFF12377DD21722786676B3
:102646000008E4F608F608F608F6201A0AE54345F7
:10265600424541454070030237B7D2217D227E0FA5
:102666007F02121CB2C203C20478D2761E122BEC71
:1026760040030227E5123052AC4BAD4AAE49AF4893
:10268600A83FA93EAA3DAB3C740712033A70051257
:1026960003DD80031203EE786B120DEA78BEE69036
:1026A600487193F8E4F9FAFB740F12033A7005D2F5
:1026B6000302274C78D6120E24A83FA93EAA3DABAA
:1026C6003C1203CDA84BA94AAA49AB48740B120386
:1026D6003A702078D6120E24A83FA93EAA3DAB3CFC
:1026E6001203CD120319A84BA94AAA49AB481203F3
:1026F600CD801B78D6120E24A83FA93EAA3DAB3C3E
:102706001203CDA84BA94AAA49AB481203DD786B40
:10271600120DEA78BEE693F8E4F9FAFB740F120399
:102726003A7002D20378D6120E24A83FA93EAA3DDB
:10273600AB3C1203CDA84BA94AAA49AB4874071271
:10274600033A7002D2033004030227E5786606E6F0
:1027560024F550030227E5AC4BAD4AAE49AF480815
:1027660012042F18E6B40A77E4F9FAFB780A120283
:10277600DA7867120DEAD20478667600AC4BAD4A79
:10278600AE49AF48A83FA93EAA3DAB3C740312032D
:102796003A701A120DB47867120E24120DC612037F
:1027A600DD8C478D468E458F44C20D8018120DB4C0
:1027B6007867120E24120DC61203EE8C478D468ED4
:1027C600458F44D20DC200AC47AD46AE45AF44126C
:1027D60030B58C478D468E458F447C7012377D30E0
:1027E600042A78D206E624CD501D7600786606E6E1
:1027F60030E008122A3B122A668003121C9678667D
:10280600E624EB5002D2037C0112377D200303023B
:07281600267378D276002240
:100EEA0044454C2D414C0020452D44454C00205092
:100EFA002D4F4E200020502D4F4646002053756D31
:100F0A0020546F74616C202000286C62290020280C
:0F0F1A00672900286B67290020484F4C442000AE
:10281D003232323278A490488F790E120D86D2A6BC
:10282D007C0F12377D121C8975260012374FC2A6F8
:10283D0078D27600752B00752A00121E70C20CC25C
:10284D0020C21130950302291A30950302291A78F6
:10285D00A2760078A2E624F9401AE6540175F00735
:10286D00A424A4FDE4FEFF121CB27C7F12377D78F8
:10287D00A20680DFD20A123D121220E6400280F934
:10288D0012214A78A3ECF6700E123D3DECB405050D
:10289D00123D6C80EB80E97C401237A1C2AC78A36D
:1028AD00E6120B85000C290B28CF28E428E428E438
:1028BD0028E928E428EF28E428F128F6290B28FB3D
:1028CD0029007D297E0F7F02121CB27C1012377DEC
:1028DD00121E70C20A80291242688024C312441C41
:1028ED00801E801C12461080171218AD80121242E5
:1028FD00CD800DD2201210E75002C20A8002800056
:10290D00121C89D2AC300A03022886C2AC20950B6A
:10291D007D307E0F7F02121CB280F220950B7D3030
:10292D007E0F7F02121CB280F2120FF81237E012E6
:10293D003516E52830E715D21830450E7D377E0F58
:10294D007F02121CB27CFF12377D8013C2183045F6
:10295D000E7D3E7E0F7F02121CB27CFF12377D78FA
:10296D00D37600C20FC216C21CD217C21BC214C22C
:10297D0012C215C21EC21FC20DC21AC210C219C286
:10298D0021C222C227C223C224C213E4F54FF54E41
:10299D00F54DF54C78D6F608F608F608F678D376A8
:1029AD000078D4760078D57600F547F546F545F5EF
:1029BD0044F543F542F541F5401234F07C60123791
:1029CD00A1123D12122BEC5008122D6D122A3B80D4
:1029DD0055123EBA78A27600301E091220E650023A
:1029ED00C21E80E012214A78A3ECF6700280D57CDD
:1029FD00401237A1C2AC78A3E624F418F624FC509B
:102A0D00027604E625E024CDF582E43447F583E42F
:102A1D0093FD740193F5828D83120E5C120E69D2B3
:102A2D00AC300C028005122A66809902282B301BCF
:102A3D001D7D457E0F7F02121CB21237B77CFF122F
:102A4D00377D78D47600C20F78D37600800A122AAB
:102A5D0066AC43AD42121CE722C202AC4BAD4AAE8E
:102A6D0049AF48A83FA93EAA3DAB3C740712033AB3
:102A7D0070051203DD80031203EE7862120DEA7801
:102A8D0060760130150E78BEE69048719378602619
:102A9D0008F6800D78BEE690487193C3786096086D
:102AAD00F6C215FCE4FDFEFF08120E30740312038E
:102ABD003A701BD21578D6E6084608460846700BC4
:102ACD00C20DE4F547F546F545F544022B8778D65A
:102ADD00E60846084608467003022B6D78D6120E9E
:102AED0024A83FA93EAA3DAB3C1203CDA84BA94A51
:102AFD00AA49AB48740B12033A702078D6120E24F3
:102B0D00A83FA93EAA3DAB3C1203CD120319A84B19
:102B1D00A94AAA49AB481203CD801B78D6120E24C0
:102B2D00A83FA93EAA3DAB3C1203CDA84BA94AAA8A
:102B3D0049AB481203DD7862120DEA7861E6F8E4DC
:102B4D00F9FAFB740F12033A7016D215C20DC200BA
:102B5D0078D6120E241230B58C478D468E458F4493
:102B6D0078BEE690488993FCE4FDFEFF7862120E74
:102B7D0030740B12033A7002D202C20078D6120ED4
:102B8D00241230B57862120DEA300D25A847A946FA
:102B9D00AA45AB441203CD8C438D428E418F40E547
:102BAD004345424541454060027401A2E0921A80BE
:102BBD002BA847A946AA45AB44740F12033A700FD0
:102BCD001203EE8C438D428E418F40C21A800D123E
:102BDD0003DD8C438D428E418F40D21A0234F0308A
:102BED00B32CE52B2473502078CBE604F6600280DD
:102BFD00157D4C7E0F7F02121CB280FE7CFF1237BA
:102C0D007D7CFF12377D800478CB7600804178CBB8
:102C1D00E6703C04F6AC8DE4FDFEFF78081203AAC5
:102C2D00A88BE4F9FAFB1203CD8C4B8D4A8E498F9C
:102C3D004830250B7848E4FCFDFF04FE12042F30CC
:102C4D008F0B7848E4FCFDFF04FE12042FD322C342
:102C5D0022C205AC4BAD4AAE49AF48A83FA93EAA2A
:102C6D003DAB3C740712033A70051203DD8003126D
:102C7D0003EE7870120DEA78BEE690488393F8E47F
:102C8D00F9FAFB740F12033A7006D205C206807E64
:102C9D0078D6E6084608460846607378D6120E24A4
:102CAD00A83FA93EAA3DAB3C1203CDA84BA94AAA09
:102CBD0049AB48740B12033A702078D6120E24A833
:102CCD003FA93EAA3DAB3C1203CD120319A84BA957
:102CDD004AAA49AB481203CD801B78D6120E24A800
:102CED003FA93EAA3DAB3C1203CDA84BA94AAA4928
:102CFD00AB481203DD7870120DEA78BEE693F8E466
:102D0D00F9FAFB740F12033A7004D205D206EC4D9A
:102D1D004E4F70012230051778D306E624F8500B7C
:102D2D00D2017C0212365F92058002C205800478C2
:102D3D00D3760030052978D3760030061278D61276
:102D4D000E24A84BA94AAA49AB481203EE8008AC41
:102D5D004BAD4AAE49AF488C3F8D3E8E3D8F3C22E8
:102D6D0078D2E6600214F6E5275407904863937510
:102D7D00F005A4ADF0FCED3395E0FEFFA843A942AC
:102D8D00AA41AB40740F12033A7050E527540793D4
:102D9D0075F005A4ADF078D126FC18ED36FDE4FEF6
:102DAD00FFA843A942AA41AB40740312033A702B0A
:102DBD00E52754079375F005A4ADF0FCC3E49CFC26
:102DCD00E49DFD78D1EC26FC18ED36FDA843A94213
:102DDD00AA41AB40740712033A7008D20178D0E4CF
:102DED00F608F678747603123052E54B454A45499C
:102DFD004548701D787416B6000E7D4C7E0F7F020F
:102E0D00121CB27CFE02377D122BEC400280F98041
:102E1D0004787476007874E670CDAC4BAD4AAE494B
:102E2D00AF48A84FA94EAA4DAB4C740712033A7088
:102E3D00051203DD80031203EE7875120DEA300FD3
:102E4D005C7874760AE52830E3027619E6FCE4FD39
:102E5D00FEFF08120E30740B12033A701078D47600
:102E6D000078D37600C20F78D57600802E78D506FF
:102E7D00E624F8502678BEE690488393FCE4FDFEE8
:102E8D00FF7875120E30740B12033A700A78D476EF
:102E9D000078D37600C20F78D57600802C78BEE608
:102EAD0090486B93FCE4FDFEFF7875120E307403B1
:102EBD0012033A700E78D4E624FE4003068002D247
:102ECD000F800678D47600C20F300F4A78D2E670A4
:102EDD0033300130E52754079048639375F005A40E
:102EED00ADF0FCED3395E0FEFFA843A942AA41AB3E
:102EFD0040740B12033A700C12384D78D0A642086C
:102F0D00A643C20130160F30150CE543454245412D
:102F1D0045407002C21678D2E67006304003123872
:102F2D004D300F11C207122C5E78D4E624FB400100
:102F3D00227600800478D37600854B4F854A4E85E6
:102F4D00494D85484CAC4BAD4AAE49AF48A83FA959
:102F5D003EAA3DAB3C740312033A700F1203DD8C95
:102F6D00478D468E458F44C20D800D1203EE8C4762
:102F7D008D468E458F44D20DE527C4030354037847
:102F8D0074F6B4031A7E027D807C07121FDD78C3B0
:102F9D00E6FD08E6FCE4FEFF7875120DEA806FFC95
:102FAD0025E025E0244FF582E43448F583120E4CDC
:102FBD00E87875120E02E5270303035407FC7874B5
:102FCD00F6B4070D08E4FEFF04FD7CD612042F8035
:102FDD003DB4061908E4FEFF04FD7CD612042F3023
:102FED003A09E4FDFEFF7C5A120449802190485BAA
:102FFD009375F00384FEEC9375F009A4ABF0FAEE33
:10300D002AFCE43BFD3395E0FEFF0812042FAC478C
:10301D00AD46AE45AF447875120E30740712033AC3
:10302D007007D21B121C898002C21BA21B9214C2F4
:10303D0000AC47AD46AE45AF441230B58C478D461A
:10304D008E458F4422AC4BAD4AAE49AF4812098F25
:10305D007852120DEAA82FA92EAA2DAB2C1205819C
:10306D007852120E30120581120DA27852120E24D2
:10307D00A833A932AA31AB30120581120DC6120840
:10308D0033A837A936AA35AB341208337856120D4A
:10309D00EAA83BA93AAA39AB381205811209308C3E
:1030AD004B8D4A8E498F4822E52703030354077839
:1030BD0052F6E527540708F6785C120DEA30000346
:1030CD0002315478D6E608460846084660677854BB
:1030DD00E4F608F608F608F608F608F608F608F617
:1030ED0078D6120E24A83FA93EAA3DAB3C1203CDC3
:1030FD00A84BA94AAA49AB48740312033A702A781F
:10310D00D6120E24A83FA93EAA3DAB3C1203CDA872
:10311D004BA94AAA49AB481203DD785C120E301256
:10312D0003DD7858120DEA800A78D6120E247854F1
:10313D00120DEA80127854E4F608F608F608F6083F
:10314D00F608F608F608F67852E6B4070280030290
:10315D003234A23882395042785C120E24785812DB
:10316D000E301203CD120DA27854120E24E4FB047E
:10317D00FA792478F81203CD120DC6740312033AAE
:10318D00700D78BE76027852760308760280087844
:10319D00BE760478527605023234303841785C12AE
:1031AD000E247858120E301203CD120DA27854123F
:1031BD000E24E4FB04FA792478F81203CD120DC61F
:1031CD00740312033A700D78BE76027852760308B6
:1031DD007600800878BE76047852760580493039BD
:1031ED0040785C120E247858120E301203CD120D59
:1031FD00A27854120E24E4FAFB786079EA1203CD1A
:10320D00120DC6740312033A700D78BE7601785212
:10321D007602087601800878BE76047852760580AD
:10322D0006203A030876047852E6B40602800302BB
:10323D003471A238823940030232FE785C120E24BA
:10324D007858120E301203CD120DA27854120E249E
:10325D00E4FAFB783079751203CD120DC6740312A2
:10326D00033A703030241078BE7604E52754077881
:10327D0053F6187605801B30230D78BE76027852F2
:10328D007603087602800B78BE76007852760108B8
:10329D007601805A785C120E247858120E30120383
:1032AD00CD120DA27854120E24E4FB04FA79247881
:1032BD00F81203CD120DC6740312033A7024302494
:1032CD001078BE7604E52754077853F618760580F6
:1032DD000F78BE7602D223C2247852760308760286
:1032ED00800C78BE7604C223D2247852760502343F
:1032FD0071203A030233B9785C120E247858120EFD
:10330D00301203CD120DA27854120E24E4FAFB787C
:10331D003079751203CD120DC6740312033A703055
:10332D0030241078BE7603E52754077853F61876C7
:10333D0004801B30230D78BE760178527602087614
:10334D0003800B78BE76007852760108760280599C
:10335D00785C120E247858120E301203CD120DA285
:10336D007854120E24E4FAFB786079EA1203CD1238
:10337D000DC6740312033A702430241078BE760300
:10338D00E52754077853F6187604800F78BE76013A
:10339D00D223C22478527602087603800C78BE764A
:1033AD0003C223D2247852760402347120390302E9
:1033BD003471785C120E247858120E301203CD122F
:1033CD000DA27854120E24E4FAFB783079751203AD
:1033DD00CD120DC6740312033A703030241078BE2E
:1033ED007604E52754077853F6187605801B3023AD
:1033FD000D78BE760178527602087601800B78BE84
:10340D007600785276010876008059785C120E2489
:10341D007858120E301203CD120DA27854120E24CC
:10342D00E4FAFB786079EA1203CD120DC67403122B
:10343D00033A702430241078BE7604E527540778BB
:10344D0053F6187605800F78BE7601D223C2247804
:10345D00527602087601800C78BE7604C223D224FF
:10346D007852760578BEE690487D93FCE4FDFEFF2C
:10347D00785C12042F7852E690485B93FCE4FDFED5
:10348D00FF785C1204697853E690486393FCE4FD81
:10349D00FEFF785C02046478B8E67852F692007804
:1034AD00B9E620E3113000087852C654FEF68006C6
:1034BD007852C64401F67852E678B8F62278B8E626
:1034CD007852F6920078B9E620E311300008785270
:1034DD00C654F7F680067852C64408F67852E67858
:1034ED00B8F622A2151234A478D9E6184618461853
:1034FD00467003E480027401A2E09201301B05E4E2
:10350D00A2E09201A2E00234CAC205E527C403037A
:10351D0054037870F6FC25E025E0244FF582E43461
:10352D0048F583120E4CE4FDFEFF7C0A1202407832
:10353D0075120DEAC2001230B5C206E4F54FF54E14
:10354D00F54DF54C787076007875120DEA122BEC6E
:10355D004003023632123052E54F454E454D454C33
:10356D00700C854B4F854A4E85494D85484CAC4B6B
:10357D00AD4AAE49AF48A84FA94EAA4DAB4C740702
:10358D0012033A70051203DD80031203EE787112F7
:10359D000DEA78BEE690486B93F8E4F9FAFB740FE8
:1035AD0012033A70107870E624FD4003068004D2B1
:1035BD000676008019C20678707600E54F454E45B7
:1035CD004D454C60097D537E0F7F02121CB2854B19
:1035DD004F854A4E85494D85484C300648AC4BAD1C
:1035ED004AAE49AF4878BF120E30740712033A70D5
:1035FD00051203DD80031203EE7871120DEAC2008D
:10360D001230B57871120DEA08120E3074071203DC
:10361D003A700E7D5A7E0F7F02121CB21237B780A0
:10362D0002D205C20620050302355A121C8978BF45
:10363D00A64808A64908A64A08A64B854B3F854AC9
:10364D003E85493D85483C7875E4F608F608F60850
:10365D00F622E527C403035403786B760008760041
:10366D000876750876307862F6786FCCF6CCB403B0
:10367D001A7E027D807C07121FDD78C3E6FD08E609
:10368D00FCE4FEFF786B120DEA801525E025E024A1
:10369D004FF582E43448F583120E3C786B120DEA37
:1036AD0008E6FCE4FDFEFF786B120E301201B6E465
:1036BD00F9FAFB7864120243786B120DEAC20078B6
:1036CD006B120E241230B5786B120DEA78D6E6081F
:1036DD004608460846601278D6120E24A84BA94A11
:1036ED00AA49AB481203EE8008AC4BAD4AAE49AFC8
:1036FD00487867120DEA78BF120E30740712033A3C
:10370D00700A1203DD7863120DEA80081203EE7859
:10371D0063120DEAC2007863120E241230B578637D
:10372D00120DEA786B120E30740712033A701120E5
:10373D00010C7D5A7E0F7F02121CB21237B7C322C5
:10374D00D322758E02758CFC758A207589917588CA
:10375D001075CBFF75CAB875CDFF75CCB875C83C63
:10376D0075985043878075B80275A88275A0FF22A1
:10377D007854ECF618E6FF7E00EE04600F7F00EF44
:10378D00C378549650030F80F60E80ED7852EEF606
:10379D0008EFF622C294752A007852ECF6E52AC39A
:1037AD00785296500280F6D294227F00EF24FB408F
:1037BD001DC294752A00E52A24C4400280F8D294D3
:1037CD00752A00E52A249C400280F80F80DE78528D
:1037DD00EFF62278B27A07E4F608DAFC7A077CFF76
:1037ED0012377D7CFF12377D787176007871E62473
:1037FD00F640297F00EF24F940147871E6F4241A7D
:10380D0090481493FCEF24B2F8ECF60F80E7787033
:10381D00EFF67CAF12377D78710680D0121C897C53
:10382D007F12377D7D617E0F7F02121CB27CFF12ED
:10383D00377D7D297E0F7F02121CB27C7F02377D82
:100F2900202020202020004552522D303200205010
:100F39004F554E4400204D4554524300302D4C4FDF
:100F49004144004552522D313000554E5354424CC4
:0F0F5900004552522D30310020204144482000E5
:1047CD000E820E8E0E8A0E860E925051525354C08A
:1047DD00F9A4B0999282D880908883C6A1868E80E4
:1047ED00402010080402010102040810204080FF3F
:1047FD00FFFFFFFFFFEFFFFEFDFBF7EFDFFFFFFF0B
:10480D00FFFFFFFFFFFFDFFF40FF79246465666751
:10481D00FFFFFFDFBF7FFFC0F9A4B0999282D88060
:10482D0090B88FD4B74800888883C6A1868E9089AA
:10483D00FBF2F3C7AAABA38C98AF9287C1E3E2B6A4
:10484D0091A4000249F00001D4C0000186A0050A20
:10485D001419280814140102050A14141414091348
:10486D00182731040306070B0D020A141928320507
:10487D00050A0D14190204090B1217020812172646
:10488D002F04202043414C200020202020202000F8
:0300030002281DB3
:0300130002281EA2
:03001B0002281F99
:03002B0002282088
:040E7400000000007A
:0A0E78000000000000000000000070
:10384D002042030238FFD2AC123937D211A21A929C
:10385D0005C21A7866760B78CCE6FCE4FDFEFF1205
:10386D003BD4A205921AC2117C057D687E0F7F02A2
:10387D00123AD37866760BAC43AD42AE41AF4012EF
:10388D003BD47C01123BB578BAE60846084608469B
:10389D007002C228A21A202801B3500FAC43AD42CA
:1038AD00AE41AF4078BA12042F803978BA120E2487
:1038BD00A843A942AA41AB40740B12033A7004A26B
:1038CD001A922878BA120E24A843A942AA41AB40F5
:1038DD00740712033A70051203DD80031203EE78AC
:1038ED00BA120DEAC2AC78CC06E6B4FB037401F64D
:1038FD008037D2AC2040031239A420400B7C0B7DC5
:10390D006E7E0F7F02123AD37866760BAC43AD42D2
:10391D00AE41AF40123BD47C061239BE7C01123B46
:10392D00B5204003123A96C2AC223017697C0212C0
:10393D003BB578BAE4F608F608F608F678CC7601C9
:10394D007C097D7A7E0F7F02123AD37C057D687EDD
:10395D000F7F02123AD37C077D847E0F7F02123ACD
:10396D00D330180D7C027D8C7E0F7F02123AD380EE
:10397D001B30440D7C017D8F7E0F7F02123AD38068
:10398D000B7C027D917E0F7F02123AD37C01123B9C
:10399D00B5123A96C217227C02123BB57C0F7D946C
:1039AD007E0F7F02123AD3C2117C01123BB5023A4F
:1039BD00967870ECF678B9E654C0B44002800302F4
:1039CD003A80EC120B8500083A7C39E939FB3A0C48
:1039DD003A273A383A723A643A6B3A497C0A123BC2
:1039ED00B57C1B123B037C6D123B03023A7E7C0AB5
:1039FD00123BB57C1B123B037C69123B0380727C2E
:103A0D001B123B037C70123B037C01123B037C6455
:103A1D00123B037C90123B0380577C1B123B037CB3
:103A2D0072123B037C01123B0380467C1B123B034D
:103A3D007C72123B037C00123B0380357C1B123BD6
:103A4D00037C44123B037C08123B037C16123B03A0
:103A5D007C00123B03801A7C09123B0380137C0906
:103A6D00123B03800C7C1B123B037C40123B0380FA
:103A7D00008015ECC39406400DB40200B340077DE1
:103A8D00027C20123AB380002278B9E654C0B440CB
:103A9D00097D1E7C2D123AB380077D1A7C2D123ABA
:103AAD00B37C01023BB5785976000808EDF618ECA9
:103ABD00F67859E6C3080896500B18E6FC123B033E
:103ACD0078590680EC2278597600785DECF6785AB4
:103ADD00120DD87859E6C3785D965019785A120EA2
:103AED0012120BE4FC123B03785C06E6187001061B
:103AFD0018180680DE227858ECF678B9E654C070B6
:103B0D0042123D2F7C0412377D7C0412377D123D0D
:103B1D003D7857ECF6B41529123D3D7857ECF66417
:103B2D0006601E1806E6249B500B7DA47E0F7F02B7
:103B3D00121CB2800C7C0412377D7C0412377D8000
:103B4D00D78064B440467858E6FC123D2F7C0112B4
:103B5D00377D7C0112377D123D3D7857ECF6B4135D
:103B6D0029123D3D7857ECF66411601E1806E624C7
:103B7D0091500B7DA47E0F7F02121CB2800C7C062F
:103B8D0012377D7C0612377D80D7801BB480028072
:103B9D0003B4C0007858E6FC123D2F7C0712377D28
:103BAD007C0712377D8000227859760008ECF67874
:103BBD0059E6C30896500F7C0D123B037C0A123B4D
:103BCD000378590680E9227862120DEA08E6B40BF3
:103BDD001E301103E4800378B9E67859F6A21A5025
:103BED0004742D800274200808F6E6FC123B03785D
:103BFD0059E654079047D793540FF42406785DF691
:103C0D00C200C2017862120E2412098F785E120D65
:103C1D00EA785976007859E624FA5003023CB6E664
:103C2D0025E025E024B5F582E43447F583120E3CFA
:103C3D00785E120E301206F3120930785AECF61235
:103C4D00097218E625E025E024B5F582E43447F540
:103C5D0083120E4C120581785E120A8A7859E67825
:103C6D005D66700BD2007859E624FB4002D201202C
:103C7D000005785AE6600F785AE624300808F620D9
:103C8D000002D200800408087620785CE6FC123B26
:103C9D0003785BE6795C6719F7300107C201087696
:0E3CAD002E80E7181806023C220808E6FC22CA
:100F68002020202020002020576569676874203AD7
:100F7800200020202020436F756E74005765696734
:100F880068742F006C620067006B6700202A2A20B3
:100F9800576569676874204D6F6465004552522D26
:030FA800323000E4
:103CBB00C0E0C0D0E8C0E0ECC0E030983FC29878DC
:103CCB0051A69978CFE624F8500BD0E0FCD0E0F861
:103CDB00D0D0D0E03278CEE6B4070C7851E678C479
:103CEB00F678CE760080127851E6FC78CEE6F42496
:103CFB00C42408F8ECF678CE0678CF06D0E0FCD0DA
:103D0B00E0F8D0D0D0E03278C37A0874FFF608DA46
:103D1B00FC7A08C2AC78CD760078CE760078CF7678
:103D2B0000D2AC228C997852ECF620990280FBC21F
:103D3B009922C2AC78CFE67005D2AC7CFF2278CD4D
:103D4B00E6F424C42408F8E67852F678CF1678CD3A
:103D5B00E6B40704E4F6800204F6D2AC7852E6FC33
:103D6B0022121C897DAB7E0F7F02121CB27C0612C5
:103D7B003D2F78807600123D3D7881ECF604601A79
:103D8B0018E670060808ECF6800D1470067883ECC4
:103D9B00F680047884ECF67880067880E624FD5073
:103DAB00D5123D3DEC6406600280F67882E6FC128B
:103DBB003D2F7C0F12377D7883E6FC123D2F7C0F55
:103DCB0012377D7884E6FC123D2F7C0F12377D1263
:103DDB003D3D7881ECF604700280F4EC64036009DD
:103DEB00ECB406028003023EB6C2AC7884E678C31C
:103DFB00F67882E66405603208E654F0B4C01FE63C
:103E0B00540F44A0F6FD18E6FC7E01121FB978830F
:103E1B00E62410FD18E6FC7E01121FB9800AE6FDB0
:103E2B0018E6FC7E01121FB98051E6FC08E6FD7E08
:103E3B0001121FB97883E62440FD18E6FC7E0112BF
:103E4B001FB97883E62480FD18E6FC7E01121FB9AA
:103E5B007884E624E05024E624C4401FE624E025C1
:103E6B00E025E078C3760008760008760008760037
:103E7B007885F6FD7E047C04121FB97881E6B403C5
:103E8B0028121B7C121C897DB27E0F7F02121CB282
:103E9B007CFF1237A17C0312377D7DB97E0F7F0229
:103EAB00121CB2121E70D2AC22D2AC023D7822127E
:103EBB003D3D7879ECF6787D7600301C31B4442B9F
:103ECB00121C89C2AC7E187D007C0712400A7E1042
:103EDB007D187C0712400A7E0C7D507C0712400A2D
:103EEB007E187D307C0712400AD2AC024009047068
:103EFB0003024009201303023FFEECB411028003BE
:103F0B00023FE97C01123D2F7C02123D2F300F0D39
:103F1B007C53123D2F787DC66453F6800B7C551273
:103F2B003D2F787DC66455F6301B25787AE4F6086C
:103F3B00F6C3787BE6940718E664809480500F7C78
:103F4B0046123D2F787B06E61870010680E3802B26
:103F5B0078B9E65407787CF6700B7C20123D2F78ED
:103F6B007DC66420F67866760BAC43AD42AE41AFAE
:103F7B0040123BD4787DE66C797DF73018187C6C59
:103F8B00123D2F787DC6646CF67C62123D2F787DD6
:103F9B00C66462F680312044187C6B123D2F787D0D
:103FAB00C6646BF67C67123D2F787DC66467F6801E
:103FBB00167C20123D2F787DC66420F67C67123D5F
:103FCB002F787DC66467F6E6FC123D2F7C03123D0D
:103FDB002F7C04123D2FC213787D76008013B41210
:103FEB0009C2137C15123D2F8007C2137C15123D9D
:103FFB002F800BECB40507D2137C06123D2F22C287
:10400B0007787176007878EEF618EDF618ECF678FE
:10401B0071E6787726FD18E6FC7E01121FDD78C36A
:10402B00E67872F630072178B676FF24DF501378E6
:10403B0072E624A5400CE624E09048149378B7F67A
:10404B00800478B776FF8031FCC4540FFDEC540F1D
:10405B000808F6D206C20518EDF624F050047D0FC1
:10406B00EDF608E624F05002760FED9047DC9378DE
:10407B00B6F67874E69378B7F61221C37875ECF63A
:10408B007C601237A17875E6B40A04D205806FB450
:10409B000D04D2058068B40B17D205B2077872767F
:1040AB0020300706D31234A48004C31234A4804EEC
:1040BB00B40E04C30234A430072E24E4500DE624BE
:1040CB00CA4008E624257872F6801BE624F64008E1
:1040DB00E624307872F6800EE6B437067872762DC9
:1040EB00800478727620801654F06006E6240A5419
:1040FB000FF6300606E61818F68003E618F63007BA
:10410B001E7872E624DF5011E624A5400CE624E06D
:10411B009048149378B7F6800478B776FF802DB269
:10412B00067873E6C454F008261818F608E624F04F
:10413B005002760F08E624F05002760F18E69047EF
:10414B00DC9378B6F67874E69378B7F6200503021D
:10415B0040847872E678C3F67871E6787726FD1896
:10416B00E6FC7E01121FB97875E6B40A0E7871E68B
:10417B00C37878965003787106800AB40D0778716E
:10418B00E6600214F67871E6C37878965003024025
:10419B001AC30234A4121C897DC07E0F7F02121C2D
:1041AB00B27C06123D2F78637600123D3D7864ECAD
:1041BB00F604601A18E670060808ECF6800D147009
:1041CB00067866ECF680047867ECF678630678631D
:1041DB00E624FD50D5123D3DEC6406600280F67876
:1041EB0065E6FC123D2F7C0F12377D7866E6FC12DC
:1041FB003D2F7C0F12377D7867E6FC123D2F7C0F2D
:10420B0012377D123D3D7864ECF604700280F4ECBD
:10421B0064036004ECB40641C2AC7867E678C3F67D
:10422B007866E6FD18E6FC7E01121FB97864E6B4E9
:10423B000325121C897DC77E0F7F02121CB27CFFE7
:10424B001237A17C0312377D7DB97E0F7F02121CC2
:0D425B00B2121E70D2AC22D2AC0241AC22D5
:100FAB002050432D4C44002020454E44200020204F
:100FBB00202020200050432D4C443200444E2D4520
:030FCB004E440091
:03002300023CBBE1
:10426800C2051221C37873ECF6B40A097CFF123731
:10427800A1D205804C7C601237A17873E6249C504B
:10428800027663E675F00A841818F60808E675F0F1
:104298000A84E5F018F608E6249C50027663E67571
:1042A800F00A84FCE675F00A84E5F01818CCF6CC20
:1042B800FDEC9047DC9378B6F67872EDF69378B714
:1042C800F630059E22D2ACC205C2067DCE7E0F7F97
:1042D80002121CB27CFF12377D7DD57E0F7F021241
:1042E8001CB27CFF12377D121C891220E640028026
:1042F800F912214A7873ECF6706E123D3D7872EC33
:10430800F60460627C601237A130062D7872E6757B
:10431800F064849047DC9378B5F67872C675F064DB
:1043280084E5F0F6E675F00A841818F60808E675CC
:10433800F00A84E5F018F6801478B576FF7872E60E
:10434800C4540F1818F60808E6540F18F678B27611
:10435800AF78B376B67870E69047DC9378B6F6789F
:1043680071E69378B7F68089B40A0A7CFF1237A100
:10437800D205024413B40B2D7C601237A1B206306B
:10438800060B7DDC7E0F7F02121CB280097DE37E66
:104398000F7F02121CB27CFF12377D7CFF12377D23
:1043A800121C8980667C601237A17873E6FC123D86
:1043B8002F7873E618F6300629FC75F06484904768
:1043C800DC9378B5F6EC75F06484E5F07872F6FC69
:1043D80075F00A841818F6EC75F00A84E5F008F60A
:1043E800801078B576FFFCC4540F7870F6EC540F43
:1043F80008F678B2768778B376B67870E69047DCB8
:104408009378B6F67871E69378B7F62005030242FA
:10441800F2C2AC2292067DEA7E0F7F02121CB27CA9
:10442800FF12377D121C897C4F12377D7DEA7E0F83
:104438007F02121CB27CFF12377D121C89300605E0
:104448007CFF12377D121E70787276007872E6242F
:10445800FD50030245FCE670067873A6278016B463
:1044680001067873A628800DB4020878B9E6787337
:10447800F6800280007873E6C4540FFCE6540F08F7
:1044880008F6C20518ECF624F050047C0FECF60888
:10449800E624F05002760F30062078B376FF787263
:1044A800E6049047DC9378B4F60876BFEC9378B6C8
:1044B800F67875E69378B7F6801E78B376FF78724B
:1044C800E6049047DC9378B4F60876BFEC9378B6A8
:1044D800F67875E69378B7F61221C37876ECF6305D
:1044E8000649B40C057C600237A1B40D10D20578DA
:1044F80072E624FD40057C601237A1802CB40E0FB3
:104508007C601237A17875E618F6087600801AB430
:104518000F117C601237A1787506E624F0500276F8
:104528000080061237B70245C1802EB40A10D205A2
:104538007872E624FA40057C601237A1801B7C6003
:104548001237A17876E654F06006E6240A540FF68E
:1045580018E618F60808E618F67874E6C454F00861
:10456800261818F608E624F05002760F08E624F01C
:104578005002760F30062278B376FF7872E6049000
:1045880047DC9378B4F60876BF7874E69378B6F685
:104598007875E69378B7F6802078B376FF7872E678
:1045A800049047DC9378B4F60876BF7874E693787D
:1045B800B6F67875E69378B7F62005030244E078F6
:1045C80072E670077873E6F5278017B401077873E9
:1045D800E6F528800DB402087873E678B9F680020B
:1045E80080003006097872E624FE50028006787250
:1045F80006024454121F087DF17E0F7F02121CB27E
:104608007CFF1237A1021C8978B27A07E4F608DA2F
:10461800FC7A071220E6400280F97C401237A1029A
:024628001C89EB
:100FCE0052532D32333200202054455354004445A1
:100FDE0043203130004845582031360020432D53F0
:0A0FEE004554002020454E44200029
:10462A00C292D293D292D292D292D292D292D2926F
:10463A00C293C293C293C293C293C29222C292C23B
:10464A0093D292D292D292D292D292D292D293D23E
:10465A0093D293D293D293C29222D292D292D292EC
:10466A00D292D292C292C292C292C292C29222783A
:10467A0053E6FF7E00EE24F84019D293D292D292EA
:10468A00D292D292EF25E0A29372E092E0FFC29218
:10469A000E80E27852EEF608EFF6FC22C29302464A
:1046AA0064D2930246648C297853ECF61876007823
:1046BA0052E624F84012A24F9293124664E5292545
:1046CA00E0F52978520680E7752900D29376FF3003
:1046DA00930D785216B60005752901800280F012F2
:1046EA004664AC29227857EDF618ECF612462A7879
:1046FA0056E625E0540E44A018F6FC1246B0EC60CB
:10470A000512464780E67857E6FC1246B07854769A
:10471A00007854E6C3785B9650197858120E1278CE
:10472A0054E6F582758300120BE9FC1246B0785400
:10473A000680DE0246477857EDF618ECF612462A4E
:10474A007856E625E0540E44A018F6FC1246B0EC62
:10475A00600512464780E67857E6FC1246B01246D4
:10476A002A7855C64401F6E6FC1246B0785476001B
:10477A001246797858120E127854E606F582758335
:10478A0000EC120D0C7854E6785B66700280051214
:0A479A0046A680DC1246AB0246473B
:0300000002002ECD
:10002E007581D99000018583A01247A4EC4D6051D3
:10003E0078D97600D8FC900001AE83AF8290000193
:10004E001200986005E4F0A380F6900001A982905A
:10005E000001A882E899500576000880F79000F616
:10006E001200A19000FA1200A19000FE1200A190C1
:10007E0001021200BF9001081200BF90010E120083
:10008E00BF75D000122821020114EF65827003EEB5
:10009E00658322E493F8740193F9740293FE74035A
:1000AE0093F5828E83E869700122E493F6A30880AB
:1000BE00F4E493FC740193FD740293FE740393FFB6
:1000CE00740493F8740593F5828883120098700176
:1000DE0022E493A3A883A9828C838D82F0A3AC83A0
:1000EE00AD828883898280E32A2A0E784C500E7462
:1000FE00D0DA0E7800010E820E8200010E820E8280
:06010E0000010FF80FF8DC
:0201140080FE6B
:0547A4007C017D0022F4
:07011600EEF8EFF9020121F0
:10011D00ECF8EDF9E88BF0A4C98AF0A429F9E88A86
:09012D00F0A4F8E5F029F94822DC
:07013600ECF8EDF9020147AE
:10013D00ECF8EDF9EBC9FBEAC8FAE94B7010E8C031
:10014D00F08AF084F8AAF0D0F079007B0022ECC0A0
:10015D00E0EDC0E0EEC0E07D007E007C10C3E83332
:10016D00F8E933F9ED33FDEE33FEED9AEE9B4005E4
:10017D00FEED9AFD08DCE6EDFAEEFBD0E0FED0E0F8
:07018D00FDD0E0FCE849226F
:07019400ECF8EDF90201A5F2
:10019B00ECF8EDF9EBC9FBEAC8FA120147EAF8EB08
:0301AB00F94822EE
:1001AE00ECF8EDF9EEFAEFFBEF4E4D4B4A49700DC0
:1001BE00E88CF0A4FCADF07E007F004D22C082ECF6
:1001CE00F58288F0A4C0E0E8C5F0CDC0E0A42DFD16
:1001DE00E435F0CEFC8582F0E9A42DFDEE35F0FE7F
:1001EE00E433CF88F0A42FFFE98CF0A42FFFEAD0E0
:1001FE00F0C0F0A42FFFEB8582F0A42FFFD0F0E922
:10020E00A42EFEEF35F0FFEA8582F0A42EFEEF3528
:10021E00F0FF8CF0E8A42EFEEF35F0FFD0E0D08298
:05022E00FC4E4D4F22C3
:0D023300EFCBFFEECAFEEDC9FDECC8FC22CA
:10024000120233EB4A4E4F7017ECFAEDFB120141EC
:10025000F5F0E8FCE9FDEAF8EBF9E4FAFBE5F02259
:10026000C082C08375F0208B828883E4FBCFC0E01E
:10027000E4CACEC0E0E4C9CDC0E0C3EC33FCA88141
:10028000E633F618E633F618E633F6EB33FBE933DC
:10029000F9EA33FAEF33FFEB9583E99DEA9EEF9598
:1002A00082400CFFEB9583FBE99DF9EA9EFA0CD5A1
:1002B000F0C8D0E0FDD0E0FEEBF8D0E0CFFBECD012
:1002C00083D0824D4E4F22120233120243EBFFEADB
:0702D000FEE9FDE8FC80ECF3
:1002D700120233EB33500EE4C398F8E499F9E49A29
:1002E700FAE49BFBD3EF30E708B3C0D012031980C1
:1002F70002C0D0120243D0F020F70122F5F012031A
:1003070019E5F022120233EFC0E01202DA1202CD31
:0203170080E480
:10031900E4C39CFCE49DFDE49EFEE49FFF4E4D4C2E
:0103290022B1
:10032A00ECF4FCEDF4FDEEF4FEEFF4FF4E4D4C223E
:10033A00C083F5F0C3EC98F583ED994283EE9A42B7
:10034A008320F010C082EB6480F582EF648095828E
:10035A00D0828002EF9B82F130F20545837001D38F
:09036A00D08330F301B3E4332227
:1003730088F005F0800EEFA2E713FFEE13FEED13F6
:0C038300FDEC13FCD5F0EFEF4E4D4C22CA
:10038F0088F005F0800DC3EF13FFEE13FEED13FDA4
:0B039F00EC13FCD5F0F0EF4E4D4C22AB
:1003AA0088F005F0800DC3EC33FCED33FDEE33FE2F
:0B03BA00EF33FFD5F0F0EF4E4D4C226A
:1003C500ECF8EDF9EEFAEFFBEC28FCED39FDEE3A31
:0803D500FEEF3BFF4E4D4C22F0
:1003DD00C3EC98FCED99FDEE9AFEEF9BFF4E4D4C54
:0103ED0022ED
:1003EE00C3E89CFCE99DFDEA9EFEEB9FFF4E4D4C43
:0103FE0022DC
:1003FF00EC58FCED59FDEE5AFEEF5BFF4E4D4C22D3
:10040F00EC48FCED49FDEE4AFEEF4BFF4E4D4C2202
:10041F00EC68FCED69FDEE6AFEEF6BFF4E4D4C2272
:10042F00080808E62CFCF618E63DFDF618E63EFE39
:0A043F00F618E63FFFF64E4D4C2282
:10044900080808E6C39CFCF618E69DFDF618E69E2A
:0B045900FEF618E69FFFF64E4D4C2209
:0504640075F021800885
:0504690075F041800365
:10046E0075F091EBC0E0EAC0E0E9C0E0E8C0E0ED75
:10047E00F9EEFAEFFBE6FF08E6FE08E6FD08E6CC2D
:10048E00C830F310CCC0E0CCCDC0E0CDCEC0E0CEB5
:09049E00CFC0E0CFC0E00204B2BF
:0B04A700E814600104F9FAFB0203CD29
:1004B200C0F0E5F0C4540F75F005A49004C17312A6
:1004C20003CD80491203DD80441201B6803F12023F
:1004D200DA803A120243803512030E80301202CAC9
:1004E200802B120373802612038F80211203AA80AD
:1004F2001C1203FF801712040F801212041F800DBA
:100502001204A78008120319800312032AD0F0FBF9
:1005120030F010D0E0F8ECF618EDF618EEF618EF21
:10052200F6802E30F21DD083D082EFF0A3EEF0A33E
:10053200EDF0A3ECF0E58224FDF582E58334FFF5CE
:1005420083800ED0E0F8ECF218EDF218EEF218EF1C
:10055200F230F310D0E0FFD0E0FED0E0FDD0E0FCBE
:100562004D4E4FFBD0E0F8D0E0F9D0E0FAD0E0CB2E
:010572002266
:06057300E4F8F902058125
:10057900ECF8EDF9EEFAEFFBEF4E700122EB4A7061
:1005890005FFFCFDFE221207E2947F40092B500C67
:100599007F7F74FF80EC2B4003E480E5C0E0C0F06E
:1005A900E849704EBA8009D0E0F9D0E0F80206A90E
:1005B900EC4D7018BE8008E8FCE9FDEAFE80E8E42D
:1005C900FBFFEA8EF0A4F8E5F0020675EA8CF0A4C8
:1005D900FFABF0EA8DF0A42BFBE435F0F8EA8EF0DE
:1005E900A428F8E435F0020675EACEFAE9FDE8FC3C
:1005F90080DAEC4D7005BE80F080BCEAC0E0EC8882
:10060900F0A4FFABF0ED88F0A42BFBE435F0FAEC95
:1006190089F0A42B4FFFE5F03AFAE433FB88F0EEBA
:10062900A42AFAE5F03BFBED89F0A42AFAE5F03BB0
:10063900FBE433F88CF0D0E0FCA42AC5F03BFBE4E2
:1006490038F8EF6002D2F0AFF0ED8CF0A42BFBE5A7
:10065900F038F8E433FAEE89F0A42BFBE5F038F82A
:10066900E43AFAEC8EF0A428F8E5F03AF5F0FEE861
:10067900FDEBFCD0E0F9D0E0F830F70608B800054A
:05068900802B1206C2E7
:10068E00EF3350178CF020F00260100CBC000C0DF4
:10069E00BD00080EBE000408E8600DE933E813FF44
:1006AE00EE2313FE4F4D4C227F7F74FF8002E4FF3A
:0406BE00FEFDFC221F
:0E06C200C3EF33FFEC33FCED33FDEE33FE22CD
:1006D000C3EE13FEED13FDEC13FCEF135002D2E05A
:0206E000FF22F7
:0E06E200C3E49CFCE49DFDE49EFEE49FFF2229
:1006F000E4FCFDEFCBFFEECAFEEDC9FDECC8FCEF5C
:100700004E60B9EB4A60AF1207E2EB947FCF400531
:100710009F500680A7C39F509DFBE849700CEA9448
:10072000807007EBF8A9F00206A9C0F07F0012075D
:10073000D3501EEB6002DB05D0F00206BCC31206EC
:10074000C6EF33FFEC28FCED39FDEE3AFEE43FFF47
:10075000D3EBC0E075F0087403C0E07B00501CC30D
:10076000EC98FCED99FDEE9AFEEF9400FF500CEC36
:1007700028FCED39FDEE3AFEE43FFFEB33FBEC33B2
:10078000FCED33FDEE33FEEF33FFD5F012D0F0EB8E
:10079000C0E0E5F0146012C0E075F0087B00EF20C7
:1007A000E0BDEED330E7D480B61207D34E4D4CFBFC
:1007B000D0E0F4FCD0E0F4FDD0E0F4FED0E0F8D0DE
:1007C000E0F9EB50030206A96003020699EC54011C
:1007D000020697C3EC98FCED99FDEE9AFEEF9400AB
:0207E000FF22F6
:1007E200EAA2E7D2E7FAEB33FB13F5F0EEA2E7D287
:1007F200E7FEEF33FFC5F013A2E730E601B313C5FE
:03080200F0C3221E
:09080500E8FB7A80E4F9F8802593
:09080E00ECFF7E80E4FDFC801C7F
:10081700E4FCFDEFCBFFEECAFEEDC9FDECC8FCEB37
:100827004A7003EF4E22EB6480FB8007EB4A7003AC
:10083700EF4E22EF4E700BEBFFEAFEE9FDE8FC748A
:100847000122C3EC98ED99EE9AEBC2E7F5F0EFC2FF
:10085700E795F0500E600CEBCFFBEACEFAE9CDF945
:10086700E8CCF81207E2C0E0C0F07F00C39BFB6052
:100877005B9418600C401AD0E023F9D0E0F8020628
:10088700A98AF0E9486003D2F0E4AFF0FAF9F880FA
:100897003BEB30E40D89F0EA6003D2F0E4AFF0F906
:1008A700CAF8EB30E30D88F0EF6002D2F0AFF0E466
:1008B700CAC9F8EB54076014FBC3EA13FAE913F942
:1008C700E813F8EF135002D2E0FFDBEDD0E0C0E011
:1008D70030E734C3E49FFFF5F0EC98FC42F0ED9964
:1008E700FD42F0EE9AFE42F0D0E0F9D0E0F8E5F0F4
:1008F700700122E923F9EE30E70302068ED80302DE
:1009070006BC1206C280F0EC28FCED39FDEE3AFE7B
:10091700D0E023F9D0E0F8400302068E1206D10892
:09092700B800030206B602068EB8
:10093000EF4E7003FDFC22EEA2E7D2E7FEE4CF33D8
:1009400092D5C3947F50030206BCF5F0941F400576
:1009500060110206B6F404F5F0EF54FEFF1206D063
:10096000D5F0F6EFCCCDCECF30D5031206E2EE02B5
:0209700006B2CD
:07097200FCE4FDFEFF80160E
:05097900E4FEFF801107
:10097E00ED3395E0FEFFEF30E707D2D51206E280A9
:10098E0002C2D5EF4E4D4C70012275F096EF700EEF
:10099E00EE20E71C15F01206C230E7F88012EF05C4
:1009AE00F0C313FFEE13FEED13FDEC13FCEF70EF2F
:0D09BE00A2D5E5F013FFEE92E7FE44012202
:0509CB00E4FAFB801BB3
:1009D000E93395E0FAFBEB30E711D2D5C3E498F8A0
:1009E000E499F9E49AFAE49BFB8002C2D5EB4A4908
:1009F0004870012275F096EB7018EA20E72615F092
:100A0000C3EB33FBE833F8E933F9EA33FA30E7EEC6
:100A10008012EB05F0C313FBEA13FAE913F9E813AC
:100A2000F8EB70EFA2D5E5F013FBEA92E7FA440188
:010A300022A3
:100A31007C007D00F5F0C3EF20E706EB30E7148082
:100A410034EB20E704F4D3802C30F10363F00CEB9A
:100A5100547FFBEF4E7002FCFDEB4A7002F8F9EC9B
:100A610098A8F0F5F0ED9942F0EE9A42F0EF547F3C
:100A71009B45F088F082F130F2037001D330F3012D
:040A8100B3E4332285
:050A850075F001800E78
:050A8A0075F011800968
:050A8F0075F021800458
:100A940075F049FCEBC0E0EAC0E0E9C0E0E8C0E082
:100AA400E6FB08E6FA08E6F908E6C830F310C8C021
:100AB400E0C8C9C0E0C9CAC0E0CACBC0E0CBC0E04E
:100AC400C0F0E5F0C4540F75F005A47582D67583A3
:100AD4000A73120833803A12081A8035120581808D
:100AE400301206F3802B12080E8026120B7580211B
:100AF400120833801C1208268017120581801212F6
:100B040006FF800D1208058008EF4E6004EFB2E77F
:100B1400FFD0F0FB30F010D0E0F8ECF618EDF6184A
:100B2400EEF618EFF6802E30F21DD083D082EFF06F
:100B3400A3EEF0A3EDF0A3ECF0E58224FDF582E54D
:100B44008334FFF583800ED0E0F8ECF218EDF21850
:100B5400EEF218EFF230F30CD0E0FFD0E0FED0E07C
:100B6400FDD0E0FCD0E0F8D0E0F9D0E0FAD0E0CB62
:010B7400225E
:100B7500E8FCE9FDEAFEEBFF4E6004EFB2E7FF2279
:100B8500D083D082F5F0C3E493A3C5F095F0C0E01F
:100B9500C3D0F0E493A395F04012A3A3C3E5F033CB
:100BA500500205832582F58250020583740193C0A6
:060BB500E0E493C0E02221
:100BBB00D083D082F5F0E49370097401937004A391
:100BCB00A3800C74029365F06005A3A3A380E77464
:090BDB000193C0E0E493C0E022A4
:050BE400120CBA8003B1
:030BE900120CDB10
:100BEC0030E00720E302E622E72230E10720E302AF
:0C0BFC00E222E32230E202E022E4932235
:050C0800120C898000C0
:0A0C0D00AFF0120C35CFC5F0CF2276
:050C1700120CDB80005F
:0A0C1C00A9F0120C35C9C5F0C92279
:050C2600120CDB800050
:0A0C2B00ABF0120C35CBC5F0CB2264
:100C350030E01020E306E6F5F008E622E7F5F009D6
:100C4500E7192230E11020E306E2F5F008E222E39D
:100C5500F5F009E3192230E206E0F5F0A3E022E41D
:070C650093F5F074019322E6
:100C6C00BB0003740922BB010789828A83740422A6
:0D0C7C00BB020789828A83741022740A2249
:100C8900BB0007E92582F8740122BB010DE9258221
:100C9900F582EA3583F583740422BB020DE92582C6
:100CA900F582EA3583F583741022E92582F8740206
:010CB9002218
:100CBA00BF0005EDF8740122BF01078D828E83748F
:100CCA000422BF02078D828E83741022EDF874020B
:010CDA0022F7
:100CDB00BF0007ED2582F8740122BF010DED2582BF
:100CEB00F582EE3583F583740422BF020DED258268
:100CFB00F582EE3583F583741022ED2582F87402AC
:010D0B0022C5
:050D0C00C0E0120CDB49
:100D110030E00B20E304D0E0F622D0E0F72230E10E
:100D21000B20E304D0E0F222D0E0F322D0E0F02265
:050D3100120C6C8000B3
:100D360030E01E20E30CEFF608EEF608EDF608ECC0
:100D4600F622EFF709EEF709EDF709ECF71919198D
:100D56002230E11E20E30CEFF208EEF208EDF20875
:100D6600ECF222EFF309EEF309EDF309ECF31919AE
:0E0D76001922EFF0A3EEF0A3EDF0A3ECF022B3
:080D840008A3E493F6D9F9225B
:0B0D8C0025E0F582E933F583020C1727
:0B0D970025E0F582EF33F583020C0825
:100DA200D083D082EFC0E0EEC0E0EDC0E0ECC0E066
:020DB200E473E8
:100DB400D083D082EBC0E0EAC0E0E9C0E0E8C0E064
:020DC400E473D6
:100DC600D083D082D0E0F8D0E0F9D0E0FAD0E0FBD2
:020DD600E473C4
:090DD800EFF608EEF608EDF62234
:090DE100EBF608EAF608E9F62237
:0C0DEA00EFF608EEF608EDF608ECF62235
:0C0DF600EFF709EEF709EDF709ECF72222
:100E0200C0E0EBF608EAF608E9F608D0E0F6F822C8
:090E1200E6FF08E6FE08E6FD22F9
:090E1B00E6FB08E6FA08E6F922FC
:0C0E2400E6FF08E6FE08E6FD08E6FC22FA
:0C0E3000E6FB08E6FA08E6F908E6F822FE
:100E3C00E493FF740193FE740293FD740393FC22FC
:100E4C00E493FB740193FA740293F9740393F822FC
:0D0E5C00740193F5F0E493F58385F0822294
:020E6900E47330
:090E6B00E8FCE9FDEAFEEBFF22C0
:00000001FF
:00000001FF
